:10006800102F1A951123E9F708950A93EA93FA9342
:10007800FFB7FA93E1E700810E7F008305B70F7D94
:1000880005BFF991FFBFF991E9910991189519B741
:100098001D7F19BF112713BF18B7126018BF4095ED
:1000A80042BF15B71F7E106215BFE1E710811160CE
:1000B800108319B7126019BF03BF08958895E1E747
:1000C800008100FDFCCF09B70D7F09BF08951127F6
:1000D80011BB1FEF12BB112717BB1FEF18BB08601E
:1000E80001BDA89505B7006305BF0895202F3327E4
:1000F80000270417E8F4E22F11912E2F55275830C6
:10010800A8F4632F61276170662311F06FEF01C0B7
:100118006627732F777E3627E32FE871372F3E2B1C
:1001280036956078362B16955395E9CF0395E1CF30
:10013800032F0895F2D2440F440F440F142F842F35
:1001480099270896212F3327281739075CF4E19956
:10015800FECF1EBB21E02CBB2DB3E02F03952083DF
:100168001395EDCFE2E0EAC2102F110F110F110F16
:10017800012F212F3327285F3F4F602F77276217E2
:100188007307BCF4E199FECF0EBB21E02CBB2DB365
:10019800E42F3081321751F0E199FECF0EBBE42FE6
:1001A80020812DBB24E02CBB22E02CBB439503957A
:1001B800E0CF0895B1D2802F982F913310F09A3361
:1001C80088F0903311F49AE00DC09D3211F49FE04D
:1001D80009C0903511F49EE005C0963411F49BE0F7
:1001E80001C09927F894A8E0AA2389F0BC9802E0F6
:1001F80037DF092F0A23002311F0BB9801C0BB9AEF
:1002080003E02EDFBC9A04E02BDFA695EDCF7894AF
:10021800082FE3E092C28A938AE000E2CBDF8A9556
:100228008823D9F7899108958A93802FE82F008130
:10023800002329F0E82F01918E2FBCDFF7CF899199
:1002480008958A93802F00272227843618F0845631
:100258000395FBCF002319F0005DACDF2FEF0027DB
:100268008A3018F08A500395FBCF102F122B1123D8
:1002780011F0005D9FDF082F005D9CDF89910895D4
:100288008A93802F803034F40DE294DF0027081B16
:10029800D8DF02C0082FD5DF899108958B9A02E034
:1002A800DFDE829B02C00027089501E008958B9845
:1002B80008958A9A4CEE02E0EADE00DF8A984CEE56
:1002C80002E0E5DEFBDE08958A93802FF8948A9A8F
:1002D80002E0C6DE882309F08A98789448EB01E0AA
:1002E800D6DEECDE8A98899108958A93F8948A9AE2
:1002F80002E0B6DE8A980CE0B3DE829B02C08FEF84
:1003080001C08827789444E801E0C1DED7DE082FD1
:100318008991089502D2802F91E0992329F0082F1E
:100328000923D2DF990FF9CFE2E008C2F6D1882776
:1003380091E0992329F0D9DF0923802B990FF9CF70
:10034800082FE2E0FBC1E9D1802F882319F40CECD7
:10035800E1DF0BC005E5DEDF98E0992331F0E82FF7
:1003680001918E2FD7DF9A95F8CFE2E0E7C1D0D17F
:100378000FEF602E5524BFEF09E6402E9ADF00EFFD
:10038800C9DF80E4A1E0E42D9081AFDF002349F0CC
:10039800ACDF002311F0002740C001E095DF9A2B65
:1003A80022C0A3DF002331F000278EDF0A2F00953B
:1003B800902319C086155CF4092F0A23002319F02D
:1003C80001E082DF10C000277FDFB82F0CC068165D
:1003D80021F401E079DF9A2B06C0002775DFB82FDA
:1003E8000A2F009590238A95AA0FAA2371F6E42D67
:1003F80043949083882331F648E009E677DE0023AA
:1004080029F449E6052DB0DE53946B2EBF3F21F049
:1004180000E1501608F4AFCF052DE7E08AC18A93B2
:10042800802F47DF082F8FDF04EB74DF5EDF8991B1
:10043800089570D1802FB42FA3E0982F3ADF0B2FA7
:1004480082DF0EEB67DF442409E0401630F46EDFEC
:10045800E92F939500834394F7CF49E0082F46DEB0
:10046800002321F00A2FAA95002339F7AA2311F0B7
:10047800002701C001E0E5E05EC14FD1902F092FB0
:10048800CEDF802F16DF092F5EDF08E443DF8823E5
:1004980021F02BDF002359F4FCCF00DF002311F0FB
:1004A80001E006C040EA04E0F2DD08DE00DF0027D4
:1004B800E2E044C131D1C950902F842FA3E0492FE5
:1004C8000C2FB7DF002311F001E032C0E82F0281C2
:1004D8001A81011729F4E82F03811B81011739F1CB
:1004E800E8DE092F30DF0EE415DFE82F028112DF86
:1004F800E82F03810FDF492F0C2F9BDF002311F01A
:1005080001E016C0E82F02811A81011729F4E82FAB
:1005180003811B81011721F00A2FAA95002301F7F7
:10052800AA2311F401E004C0092FA7DF01C00027A6
:10053800C75FE3E002C18A93842F402F082F79DF39
:10054800002311F00FEF04C0E82F048145E0BFD06D
:1005580089910895E1D0902FA42F8B81482F092FDE
:10056800EADF0A1799F0492F082F63DF002311F0FB
:1005780001E00DC00A2F45E0A5D0E82F0483482FDD
:10058800092F98DF002311F001E001C00027E4E003
:10059800D4C0C2D0A02F0A2FCEDF902F01E0492F60
:1005A80091D0902F0A2F3BDF802F83DE0A2FCBDEDE
:1005B80004E4B0DE882321F098DE002379F4FCCF30
:1005C8006DDE002311F001E00AC0990F48EB05E049
:1005D8005EDD74DD9A959923C9F769DE0027E3E0AB
:1005E800ACC08A93842F402F082F23DF002311F0FB
:1005F80005E50BC0E82F008144E069D0102FE82FF3
:10060800018144E05FD0102B012F899108950FE0FC
:1006180001BDA8958D987894002707BB002708BBD3
:10062800002701BB08E002BB00E808B98C9A0395D3
:10063800003108F00027002391F499DE902F8827D5
:10064800891768F4482F09E675DD00E60A93442700
:1006580009E680DF40E609E69CDF8A95F1CF992319
:1006680009F14A2F09E666DD40E609E6BADF802F80
:10067800853561F400E60A93442709E66BDF40E616
:1006880009E687DF40E609E6ACDF802FC4DD092FE5
:10069800D8DD02E7C9DD0A2F0395D3DD05E7C4DD00
:1006A800082FEEDDA395A91718F061DE902FAA2771
:0E06B8008C988D9A07E00BDD88950000089560
:05006200205000200009
:02000C0032C000
:020000000FC02F
:10001C0000EC05BFC7EA0FEB03500DBF4FD3002315
:10002C0009F417D0E0E6F0E002E160D3E2E6F0E09C
:10003C0000E640E04FD3E2E7F0E000E057D3E2E621
:10004C00F0E002E740E046D3E2E6F0E002E745E00C
:06005C0041D3DBD232C3E8
:0206C600FFCF64
:0406C80001E00895B0
:0A06CC004A9512F0000FE1F70895BF
:0A06D6004A9512F00695E1F7089529
:1006E000BF93AF93A02F03C0C89531960D92415090
:0806F000D8F7AF91BF91089506
:0C06F800002401C001920150E8F70895B1
:020704000000F3
:10070600FA92EA92DA92CA92BA92AA929A928A9243
:100716007A926A925A924A92BA93AA939A938A932F
:02072600089534
:10072800FF84EE84DD84CC84BB84AA849984888485
:100738007F806E805D804C80BB81AA819981888191
:0E074800F0E00FB6F894CE0FDF1F0FBE08953D
:00000001FF
